:020000040000FA
:0400000086EF00F097
:0800080000960350D8B40086F5
:10001000050E026E270E076E100E0CD8030E076E2B
:10002000E80E08D8076A640E05D8076A0A0E02D8D7
:10003000085008D0066E0950056E0850046E5DEC3D
:1000400000F00450046E024E0096035003E0025C80
:10005000D8B008D00450D8A4009600B603D0300F12
:1000600038EF00F012009EA8FED7AD6ED8801200C7
:1000700001B433EF00F001A205D001B003D001B20A
:10008000EE6E1200076A066EFF0E0626072200D0EB
:10009000D8A01200030E056EE70E02D8F5D7056A48
:1000A000FD0F046EFF0E00D001D00426000000D02A
:1000B000D8A00526D8A01200F8D7096A086A100E41
:1000C000F36E0534083609360650085C07500958A7
:1000D00005E30650085E0750095AD88004360536F5
:1000E000F32EEFD704501200A66AA68E0900F55031
:1000F00002E0EE6EFBD712004F75747075742074B9
:10010000657374206C6F6F7020232000F86A006A9A
:10011000030EAF6E200EAC6E900EAB6E400EAF6E47
:10012000900EAB6E200EAC6E0E6A0D6A0D4A0E2A52
:1001300000EE0FF0000EF76EF80EF66ED5DF020E31
:10014000016E036A0EC009F00DC008F05DDFEF6AB2
:1001500000EE0FF0EE5002E086DFFCD70D0E83DFDD
:100160000A0E81DF010E0B6E060E0B60C3EF00F06E
:1001700094928292320E86DF94928282320E82DFD5
:100180000B2AD8A4F1D709EC01F02D0E0B6E010E4D
:100190000C6E050E0C6006EF01F0949882880B50EF
:1001A00071DF94988298949A828A0B506BDF949AAC
:1001B000829A939081800B5065DF93908190939207
:1001C00081820B505FDF93928192939481840B50D4
:1001D00059DF93948194939281820B5053DF9392D1
:1001E0008192939081800B504DDF93908190949AEF
:1001F000828A0B5047DF949A829A949882880B5097
:1002000041DF949882980C2AD8A4C3D709EC01F056
:0E0210008DD78298829A8190819281941200FB
:020000040030CA
:03000100061F1FB8
:020005008385F1
:060008000FC00FE00F40E5
:00000001FF
